:100000000C9434000C9451000C9451000C94510049
:100010000C9451000C9451000C9451000C9451001C
:100020000C9451000C9451000C9451000C9451000C
:100030000C9451000C9451000C9451000C945100FC
:100040000C9451000C9451000C9451000C945100EC
:100050000C9451000C9451000C9451000C945100DC
:100060000C9451000C94510011241FBECFEFD8E026
:10007000DEBFCDBF11E0A0E0B1E0E8E0F2E002C0F9
:1000800005900D92A030B107D9F711E0A0E0B1E0E2
:1000900001C01D92A030B107E1F70E9453000C94FB
:1000A00002010C9400001F9386E284B915B88FE01A
:1000B0008AB91BB882EA8093800085E08093810032
:1000C0008FEF90E0909389008093880090938B004D
:1000D00080938A0010928500109284002D9A80E10E
:1000E00097E220E931E0F9013197F1F70197D9F76B
:1000F0002D9880E197E220E931E0F9013197F1F79D
:100100000197D9F71EE0A0E2BEE45EEF60E971E07E
:100110001AB94FEF21E030E089B182958F70482302
:10012000CD010197F1F72F5F3F4F2B303105A1F73C
:100130005AB9423021F1433018F4413049F705C033
:100140004430B9F1483021F73DC08091880090914A
:1001500089008096909389008093880080918A001E
:1001600090918B00809690938B0080938A0088E812
:1001700093E1FB013197F1F70197D9F7C9CF80914E
:1001800088009091890080979093890080938800DF
:1001900080918A0090918B00809790938B00809340
:1001A0008A0088E893E1FB013197F1F70197D9F7CD
:1001B000AFCF2D9A88E893E1FB013197F1F70197D2
:1001C000D9F7A6CF2D9888E893E1FB013197F1F795
:1001D0000197D9F79DCF8EE08AB94FEF21E030E04B
:1001E00060E27EE489B182958F704823CB0101974C
:1001F000F1F72F5F3F4F2B303105A1F78EEF8AB912
:08020000842F0895F894FFCF4C
:00000001FF
